:030000000219FDE5
:03000B000200A848
:03002B000201547B
:03005B000202DDC1
:030073000202CABC
:1000800002030406080C10182030406080040608A3
:100090000C10182030406080A0C00003070F1F051F
:1000A000050D050205030302C2AFC0D0C0E0206207
:1000B00014E5256009E473E525F4F58AD262D0E001
:1000C000D0D0D2AF3285268AC262E526F46029D02C
:1000D000E0D0D0D297D295D293D2AF32D297D295E8
:1000E000D293206F0C2066097405D5E0FDE57B42B4
:1000F00090D0E0D0D0D2AF32758A00C28DD26201EA
:10010000F101B7306805206602C29701B730680573
:10011000206602C29301B7306805206602C29501CD
:10012000B7C29630680A206607740FD5E0FDC29703
:1001300001B7C29230680A206607740FD5E0FDC28D
:100140009301B7C29430680A206607740FD5E0FDAA
:10015000C29501B7C2AFC2AD53E6EFC0D0C0E0D286
:10016000D3D2AFC2CEE52A6007207449152A21B543
:100170007800790020742EE580307E01F430E502AD
:1001800078FF53DACF207E0343DA20307E0343DA50
:1001900010C2D8C271E580307E01F430E50279FFEB
:1001A000C3E89970CB306103752A18207403752A4F
:1001B00018885CD27020740DE52B6004152B21C5C6
:1001C00043DA01C2D82070024138A85C206102C223
:1001D00070207431C3E894F0400374F0F8E8C4541C
:1001E0000F28F87984B703024105C313C31387218D
:1001F000200802C313200A06C3C898F8410528F84E
:10020000500374FFF8C3E895655003E565F888224C
:10021000E52D54066022206B1FE536C333C333F847
:10022000E564C313C313F9C3952240028922E8256C
:1002300022F52250037522FF852224A824C3E52439
:1002400095614002A8618825E5667002417CC3E89B
:10025000AA669A5003E8FAE4F9EAC333FBE568F4C6
:100260005B29400D2567F8E56760021567400B4183
:100270007C0AC3E5679A5002056778FF8826C3E5C4
:100280002594404002D26420CF0AD0E0D0D043E68B
:1002900010D2AD32C2CF053A7801E52A600530743C
:1002A00002152AC3E55C94014005755F0041C075E5
:1002B0006000756900E55F2401F55F5003755FFF1D
:1002C000D0E0D0D043E610D2AD32C2AF53E67F7556
:1002D00092FA7593FFC260759104D2AF32C2AF53E8
:1002E000E6EFC2ADC0D0C0E0C0F0D2D3D2AFA8FB21
:1002F000A9FCC2D8307102614453DACF207E034397
:10030000DA10307E0343DA20D271E580307E01F4CA
:1003100020E502611B88278928A17153DACF207E4E
:100320000343DA20307E0343DA10C2D8C27130743E
:1003300002A15D7800E580307E01F430E502A15D28
:10034000885CA14553DACF207E0343DA20307E0358
:1003500043DA10C271206102811D53DACF207E037F
:1003600043DA10307E0343DA20C2D8D2718857892D
:1003700058C3E89555F8E99556F97B007E087A0050
:10038000C3E8948CE994005005755B00810F8821C7
:1003900078A2E6A8216055C3E894C8E99400500803
:1003A000E4D2E4FB7A0A61EAC3E89468E994015074
:1003B00008E4D2E3FB7A0F61EAC3E894D0E994023F
:1003C0005008E4D2E2FB7A1E61EAC3E894A0E99403
:1003D000055008E4D2E1FB7A3C61EAC3E89498E96D
:1003E00094085008E4D2E0FB7A787E00C3E895597F
:1003F000FCE9955AFD30E70AECF42401FCEDF434F5
:1004000000FD755B00C3EC9AED9E5003755B01889F
:1004100059895A8557558558567802A145C3E8959C
:1004200027F8E99528F9307C02A129307B02A1291F
:10043000307A02A1222075028140E9FDE8FC815F4B
:10044000E9C313F9E813F8307902A122E9C313F9DB
:10045000E813F8307802A122E9C313FDE813FC2069
:10046000612CC3EC941CED940240028176ED701E69
:0F047000C3EC94C850180529E52970021529C35B
:10047F00E529940A5002A15D755C00D270A15DE57B
:10048F0029600215297888E6F97400207F0878968C
:10049F00B90302789EE624FAFEE43400FFC3EC9E13
:1004AF00FCED9FFD9208B90310A2085007207609B2
:1004BF00D27681C8307602C276A2085016B9030DE3
:1004CF00ECF42401FCEDF43400FD0204E278007931
:1004DF0000A129B90315EC33FCED33FDC3EC940AED
:1004EF00FCED9400FD50047C007D00C3EC94FFED07
:1004FF009400400678FF7900A129EC8572F0A4C51D
:10050F00F0A2F733F87900400302054578FF790030
:10051F00020545E9C313F9E813F8307C0EE96002D0
:10052F0078FFC3E81338F8E43400F9C3E894FFE91F
:10053F009400400278FF885CD270206102A15D7444
:10054F001FF4552F4BF52FC274EB7002D274752A1E
:10055F0018307403752A0A306102A1712074035395
:10056F00DAFE207403752B06D0F0D0E0D0D0D2ADD8
:10057F0043E6103279010205A179030205A1790A38
:10058F000205A1791E0205A179640205A179C802AD
:10059F0005A17817E4D5E0FDD8FAD9F6227A147BB5
:1005AF00780205C87A107B8C0205C87A0D7BB402DD
:1005BF0005C87A0B7BC80205C87902E4C292D5E060
:1005CF00FDC293D5E0FDD293D5E0FDD292D5E0FDEB
:1005DF00E920E002C29730E002C295E573D5E0FD55
:1005EF00E920E002D29730E002D2957496D5E0FD73
:1005FF00D9C9EAF8D5E0FDD8FBDBBEC29222C37C95
:10060F00007D0075F00005F0EA33FAEB33FB50F68E
:10061F00EB13FBEA13FAC3E9FFE8FEE89AF8E99B4C
:10062F00F95004EFF9EEF8B3EC33FCED33FDD5F0F0
:10063F00DFEDF9ECF822E889F08A20D2D4F8A9F09E
:10064F007B0030F70B7BFFF42401F8E9F43400F959
:10065F00E88520F0A4ADF0F8E98520F0A4AFF0FE16
:10066F00ED2EF974003FFA7C04C3EA13FAE913F98B
:10067F00E813F8DCF48BF030F70AE8F42401F8E91A
:10068F00F43400F9E889F0C2D4F8A9F02222C3E5C6
:10069F004113F9E54013F8C3E54498F8E54599F996
:1006AF00500CC3E89480E994FF40160206D4C3E8C7
:1006BF00947FE9940050030206D4787F79000206F4
:1006CF00D4788079FF8849894A22E5492546F8E59B
:1006DF004A3547F9854A20E4300701F43548FA30A6
:1006EF00E709C3EA94F04015020712C3EA940F50CA
:1006FF000302071278FF79FF7A0F02071278007949
:10070F00007AF0C3E5249561500AC3740195245013
:10071F000B020730E54A20E70E020730E54A30E7C3
:10072F0006884689478A482278A5E6FAC3E5493301
:10073F00F8E54A33F9D145E930E70BC3E89480E98E
:10074F0094FF4013E16AC3E8947FE994005002E1FB
:10075F006A787F7900E16A788079FFE820E715C32E
:10076F00E52398F84009C3E8940140030207917804
:10077F0001020791E8F424012523F84003020791B1
:10078F0078FF884B2278A6E6FAA847A948D145E911
:10079F0030E70CC3E89401E994FF40160207C5C384
:1007AF00E894FFE9940050030207C578FF7900022F
:1007BF0007C5780179FFE920E715C3E54B98F840A5
:1007CF0009C3E8940140030207EC78010207ECE843
:1007DF00F42401254BF840030207EC78FF8824220C
:1007EF0078FFC26420693D206A12D264C3E5419448
:1007FF000A4009C3E52594405002C26479A1E7601D
:10080F0023E541601F74FF8541F0848539F0306A1C
:10081F000375F005A4F8C5F0600278FFC3E895648E
:10082F005002A864886322C3E5409440E5419401D7
:10083F00E5635003140147046002F5632202084F79
:10084F002275E890227883E6FFE5E820ECF7A8BD53
:10085F00A9BE0570C3E57094084052757000E9FA9F
:0F086F0079A0E76044EA7007E571601B02088A10
:10087E00C3E895716010E5715006600C140208967D
:10088E000460F9020896E571F571C3946D401B750D
:10089E0061C0C394044013756180C39404400B750A
:1008AE006140C39404400375610075BB0822E56185
:1008BE00F460020561E570B4070375BB1022743253
:1008CE0079A787F0A4C5F0A2F733F8C3E895614085
:1008DE0002A861882288248825882688642275408B
:1008EE00007541F022C2AF75C820A8CCA9CDAA3A96
:1008FE0030CF010A75C824D2AFAB3BAC3C883B89E4
:10090E003CC3E89BF8E99C206908F930670221FF97
:10091E00215CAD3D8A3DF9EA9DFA600478FF79FFCE
:10092E00AE3EAF3F8B3E8C3FA83BA93CC3E89EF842
:10093E00E99FF9C3E54113FBE54013FAE82AF540B8
:10094E00E93BF54150067540FF7541FF21A6AA40CF
:10095E00AB41AC40AD417E047F02C3EB9404400238
:10096E001E1FC3EB940840021E1FC3ED13FDEC13B4
:10097E00FCDEF7C3EA9CFAEB9DFBEF6009C3E913BB
:10098E00F9E813F8DFF7EA28FAEB39FB8A408B41D6
:10099E0050067BFF8B408B41C3EB94025002D26713
:1009AE003069047F0321D17892E6FFC3E537948244
:1009BE0040110FC3E53794A040010FC3EF940640DA
:1009CE00027F057E02E541C4540FF9E541C454F09F
:1009DE00F8E540C4540F28F8C3E89EFAE99400FBEA
:1009EE004009C3EA9402EB940050047A02E4FB41FE
:1009FE004BAA40AB41EBC4FEEAC4540F4EFCC3EA13
:100A0E009CFAEB9400FBC3E813C313F8EA28FAEB45
:100A1E003400FB8A408B41C3EB94024002C26778DC
:100A2E0002EBC4FE7B00EAC4540F4EFAC3EA98FAF6
:100A3E004005C3940250027A027892E6FF306002BB
:100A4E00414B855192855293D26043E680C3E49A1E
:100A5E00F8E49BF930670241D7E8FAE9FBD3E913D2
:100A6E00FDE813FC88518952C3EF94036038EF20E0
:100A7E00E00DE82CF8E93DF9ECFAEDFB020AA0E8EE
:100A8E0028F8E939F9C3E82402F8E93400F97AFEC6
:100A9E007BFFC3EF9403400E8A538B54884D894ECF
:100AAE008C4F8D50610B885389548A4D8B4E8C4FD1
:100ABE008D503069127553F07554FF754FF07550A7
:100ACE00FF7551F07552FF610BE8FAD3E813FC88FD
:100ADE0051C3EF94036020EF20E007E82CF8ECFA06
:100AEE0041F7E8282402F87AFEC3EF940340088AFF
:100AFE0053884D8C4F610B88538A4D8C4FE568C3DC
:100B0E00335002646BF5683060026115753402D2A1
:100B1E006043E680E52D54066034A840A941C3E940
:100B2E0013F9E813F8C3E913F9E813F8306904E987
:100B3E002440F9C2AF53E67F759100C3E498F59453
:100B4E00E499F595759104D26043E680D2AF22D236
:100B5E0065754300752000306C03752040020B7CD8
:100B6E00D265754300752040306C03752000780106
:100B7E007901206720E52D54066002C2657914E5DF
:100B8E0041C313700104F8C3941440027814306901
:100B9E0004781B791B206010E543600C306903D587
:100BAE003404D26D811E711D0543E59B5440B52062
:100BBE0002810830690908C3E89940011861A32031
:100BCE00650A08C3E8994002617C61A3C265C2AFA1
:100BDE0053E67F7591003067127594007595FE751A
:100BEE009104D26043E680D2AF617CAE40AF41C388
:100BFE00E49EF594E49FF59561EDC3E533940150C1
:100C0E0002617C306502617CD802811C61A3C26DD9
:100C1E00C2AF53E67F7591008553948554957591B7
:100C2E0004854D92854E93D26043E680D2AFE52D7A
:100C3E0054066008206A020533020C5A306D0D20EE
:100C4E006C0A206507158115810214F02278003098
:100C5E0064053065027801E53775F007A4F9E5F013
:0F0C6E0028F5F0E9A2F013A2F113A2F213F53763
:100C7D00C394785003753778C3E53795384008D25B
:100C8D0066D297D295D2933060028194854F92852A
:100C9D005093D26043E68022207D16C2AF7542028A
:100CAD00C292D296306202C295D2AF759F13020ED8
:100CBD0094C2AF754202C292D294306202C297D2F0
:100CCD00AF759F13020E94307243207D20C2AF7515
:100CDD004203900132757B04D295C294306204C2F6
:100CED009381F2D292D2AF759F10020E94C2AF755E
:100CFD004203900132757B04D297C296306204C2D2
:100D0D0093A112D292D2AF759F11020E94207D172E
:100D1D00C2AF75420390010DD295306202C293D2DB
:100D2D00AF759F10020E94C2AF75420390010DD2A4
:100D3D0097306202C293D2AF759F11020E94207D3F
:100D4D0016C2AF754204C296D294306202C293D2DB
:100D5D00AF759F11020E94C2AF754204C294D29624
:100D6D00306202C293D2AF759F10020E943072435F
:100D7D00207D20C2AF754205900121757B40D29335
:100D8D00C292306204C297A198D296D2AF759F13CA
:100D9D00020E94C2AF754205900143757B10D2933C
:100DAD00C292306204C295A1B8D294D2AF759F138E
:100DBD00020E94207D17C2AF754205900103D293A8
:100DCD00306202C297D2AF759F13020E94C2AF75F7
:100DDD004205900117D2933062EBC295D2AF759F49
:100DED0013020E94207D16C2AF754206C294D292A4
:100DFD00306202C297D2AF759F10020E94C2AF75CA
:100E0D004206C296D292306202C295D2AF759F1140
:100E1D00020E94307243207D20C2AF7542019001C5
:100E2D0043757B10D297C296306204C295C13ED2F3
:100E3D0094D2AF759F11020E94C2AF75420190010D
:100E4D0021757B40D295C294306204C297C15ED2A7
:100E5D0096D2AF759F10020E94207D17C2AF7542CA
:100E6D0001900117D297306202C295D2AF759F11D2
:100E7D00020E94C2AF754201900103D29530620209
:100E8D00C297D2AF759F10C26622900101757B008B
:100E9D00D297D295D293C296C294C292C262227850
:100EAD008076FF0876FF0876FF0876FF0876030840
:100EBD00760408760B087601087601087601788CA1
:100ECD0076010876FF0876FF0876FF0876FF08762C
:100EDD00FF0876030876FF0876FF0876FF0876256B
:100EED000876D00876FA0876FA0876040876FF08B0
:100EFD00760108760008767A0876FF08760108767E
:100F0D0001087600087603087600227887E6FFC28E
:100F1D00727888E6C394036008C27DE630E102D2A0
:100F2D007DC27E7889E630E102D27EC3EF94026005
:100F3D0008758E01D273020F4B758E00C273227825
:100F4D0080E6149000809378A5F67881E6149000E1
:100F5D00809378A6F67886E61490008D9378A7F6A0
:100F6D007886E6F539C394025003753902789CE60C
:100F7D007538FFB402037538A0B403037538827851
:100F8D00A3E61490009A93F566D19722227896E6FF
:100F9D00FA7897E6FB7888E6B40305C3EB940EFB6D
:100FAD00307F047A007BFFC3EB9AFCC3948250021E
:100FBD007C827572000572EC8572F0A4C3E5F09425
:100FCD007D40F222D27FF19A1205927A007B007C4D
:100FDD0010120588E55C2AFA74003BFBDCF37C04F7
:100FED00C3EB13FBEA13FADCF7FEC27FF19A22E59D
:100FFD00EF20E6037520000520903FFFE5201460EB
:10100D0006901DFF1460009304600375EF1253D911
:10101D00BF7581C043FF8012058375EF0243B20394
:10102D00E5B3240220E70DF521E5E320E006852157
:10103D00B343E301120E977580FF75A40075F1B2ED
:10104D0075D4DF7590A975A5FC75F2FE75D5017582
:10105D00A60175E241120E97E4F8F6D8FD75680108
:0F106D00120EAC12154178988673753001C2AF20
:10107C0012059C1205AC1205921205B312059212C0
:10108C0005BA12059212165A12059C12059C1205ED
:10109C0097C2AF78FA79FA308507D9FBD8F7021CDA
:1010AC0000120F18120F4C120F99120F9A78988683
:1010BC0073120E9775881075890275C82475910482
:1010CC0075D84075A82275B80275E690759B807529
:1010DC009D0075D10E75BC5875BB0875BA1175E8B5
:1010EC0080120583D2AF12084C75360053DACF202C
:1010FC007E0343DA20307E0343DA1043DA01C2D890
:10110C00C27112059CD2617B037A0CE55B70077A85
:10111C000CDB0302109D12059220700302109DC27D
:10112C0070E55CC3940240E1E52F541F855E5DF5CC
:10113C005EB55DD5DAD5C26153DACF207E0343DAD2
:10114C0020307E0343DA10C2D8C27178A2E6700850
:10115C00D274E52F54E0F52FC2757529001205974E
:10116C00307409C3E529940A4002D27512058878B7
:10117C00023074027800C3E55C9840F0C2AF1205EF
:10118C00AC1205AC1205ACD2AF12059C754C0078B4
:10119C0088E6B403024180120588788CE6C394017A
:1011AC005003021280E530C39401500302128020D8
:1011BC007435C3E55C94FF5003021280C2AF120574
:1011CC00C1D2AF120597C3E55C940150EFC2AF12C8
:1011DC0005AC12058D1205ACD2AF120597C3E55CB8
:1011EC0094FF40E90216DF7F05D27F120F9A120599
:1011FC0097C2AFC27F120F9AAE5CC3E55C947FD2EC
:10120C00AF407B120583C2AF1205C1D2AFDFDA1239
:10121C000FD1C3EE94057897F612059C1215831224
:10122C0016627F0AD27F120F9A120597C2AFC27F45
:10123C00120F9AAE5CC3E55C947FD2AF50E41205FA
:10124C0083C2AF1205AC12058D1205ACD2AFDFD440
:10125C00120FD1EE24037896F612059C1215831208
:10126C001691120597120F9AC3E55C94FF50022158
:10127C00BB0216DFC3E55C954C4003855C4C120544
:10128C009778017988E7B403027805C3E55C984048
:10129C0002219BC2AF1205C11205C11205C1D2AF0A
:1012AC0012059C753000E4F531F5320531E531F469
:1012BC00703F0532789AE67819146012783214600F
:1012CC000D787D14600878FA146003753200C3E55C
:1012DC003298401D120E9712058315327531007825
:1012EC00998673C2AF1205C1D2AF78988673120576
:1012FC009712058DE52A7005307402019D78012046
:10130C0074027806C3E55C9840A17888E6C3940320
:10131C006003120597E52A700302109DC2AF120EEE
:10132C0097E4F522F523F524F525F526F567D2AFDC
:10133C007885E6C333F565E4F544F545F546F547A0
:10134C00F548F570F52CF52DF53775700875BB1053
:10135C00120583120850E5E820ECFBA8BDA9BEE9F4
:10136C007001F8887112085475700875BB10120F53
:10137C0018C2AF7561FF1208CC8522618522628587
:10138C002263D2AF752201752401752501752601E2
:10139C00856069756A017888E6B40307C27D30768A
:1013AC0002D27DD268D269753300120DF1120E2073
:1013BC001208EC1208F31208EC1208F31208EC12E3
:1013CC000B6E12069C120C5B120CA51208F3120B7E
:1013DC005D306E0312069D2067031207EF30670322
:1013EC00120836120C5B120CD41208F3120B6E306E
:1013FC006E031206D9120C5B120D4B1208F3120B72
:10140C005D306E03120737120C5B120D7A1208F363
:10141C00120B6E306E03120794120C5B120DF1124C
:10142C0008F3120850120B5D120C5B120E201208FE
:10143C00541208F330692F85646185646285606994
:10144C00756A0179187A0CC3E53399400CC269D2DC
:10145C006A8A357561FF021472C3E55C940140031E
:0F146C000213CB0214F8306A1D206C1AE53514F8
:10147B007006C26AD26B61CBF535C3E55C94014053
:10148B00030213CB0214F8753600788279A4E76057
:10149B00027803C3E55F985054307404E52A604D1D
:1014AB007888E6B40317207D0520760781C830764F
:1014BB000281C8206C07D26C856461810A78F03098
:1014CB006C058564617820C3E54198500261CB308F
:1014DB006C1BC26CC27D307602D27DD26A7535121E
:1014EB0085646161CB0536E55C600281FB75360076
:1014FB00C2AF120E977887E6FE7602120F18788726
:10150B00EEF6E4F522F523F524F525F526F56575BC
:10151B002C00752D00D2AF120597120E9778A4E60A
:10152B006006C297C293C295307409C3E536940422
:10153B004002019D41B2901A0D78201215C5E5208D
:10154B00B45A0CA31215C5E520B4A50302156312FA
:10155B000EAC121583021582901A0378807B0A1247
:10156B0015C5A308DBF9901A0F788C7B191215C5DA
:10157B00A308DBF9901A2822C2AF1216041215DE4B
:10158B00901A00740E1215CAA374061215CAA3740E
:10159B00151215CA901A0378807B0A1215C9A30875
:1015AB00DBF9901A0F788C7B191215C9A308DBF99C
:1015BB001216171215F5901A2822E493F622E64319
:1015CB008F01538FFD75EF0275B7A575B7F1F0530A
:1015DB008FFE22438F02438F0175EF0275B7A575FE
:1015EB00B7F1901A0DF0538FFC22901A0D745AB16B
:1015FB00CA901A0E74A5B1CA227A3079D07820908D
:10160B001A40B1C5E520F709A3DAF7227A3079D071
:10161B00901A40E7B1CA09A3DAF922AB74A875BBDB
:10162B0001027984BB02027985BB03027986BB0474
:10163B00027992BB05027987BB060279A3BB07022D
:10164B00799CBB08027988BB09027989E8F7227C6F
:10165B000512059CDCFB22C2AF1205AC1205B312BE
:10166B0005BA1205C112058D1205AC1205B3120590
:10167B00BA1205C112058D1205AC1205B31205BACB
:10168B001205C1D2AF22C2AF1205C11205BA1205A3
:10169B00B31205AC12058D1205C11205BA1205B3B2
:1016AB001205AC12058D1205C11205BA1205B31243
:1016BB0005ACD2AF22AE74AF75C2AF1205AC12053A
:1016CB00AC1205AC12058DDEF21205C112058DDFD1
:1016DB00F8D2AF22D162D15AD15A75740175750106
:1016EB00757600D1C07C05AD5C12059CC3ED955C95
:1016FB0070F5C3E55C9401400AC3E55C94FF40328E
:10170B0002171BD126B183D162C2AF75EF12D15A2A
:10171B00DCD50576C3E5769403500280C6D15A0515
:10172B0075E5741490009F93F808C3E57598500203
:10173B0080AED15AD15A0574C3E574940A50028015
:0D174B009C120EACB183C2AF75EF12D15AE3
:0319FD00020FFCDA
:101A00000E0615FFFFFFFF03040B0101015AA5019C
:101A1000FFFFFFFFFF03FFFFFF25D0FAFA04FF01DE
:091A2000007AFF0101000300FF40
:101A4000235475726E696779364123202020202047
:101A500023424C48454C4923463333302320202031
:101A60002020202020202020202020202020202076
:101C0000C2AFC2D353D9BF7581C043B20343FF8073
:101C1000752438752503B1C975EF0275E24043F1AB
:101C20002053A4DF75D4FFD2857DFA780379E67C52
:101C300010752200752300901DD67B0675249875BB
:101C400025013085028142208508D8FBD9F9DCF7CF
:101C500081B4308508D8FBD9F9DCF781B4B189E4C7
:101C600093A3C39A6004DDC381B4DBDBB17B600264
:101C7000812B7B08E493FAA3B15CDBF87A30B15C8A
:101C8000752200752300B17BEAFCEBFDC3ED94FEE9
:101C9000400EB17B8A278B28ED30E0048A828B834B
:101CA000B17B7AC270D8C3ED94FE601350CEBD00F4
:101CB00025EC60097520007521FF0200008100A855
:101CC00027A9280809D804D90281D3B17FEA89AAB3
:101CD000F281C50D81A0C3ED94035049EDA2E092BD
:101CE000007AC5C3E5829400E583941C50902000DF
:101CF00010438F02438F0175B7A575B7F1F030001F
:101D00001FA827A9280809438F01538FFDD804D99C
:101D100002A12089AAE275B7A575B7F1F0A3A10DBC
:101D2000538FFC817C7AC1BD030CE493A3FAB140CC
:101D3000DCF8B138817C817EAA22AB23B15CEBFA5E
:101D4000EA6222752608C3E52313F523E52213F57D
:101D50002250066323A0632201D526EAB1C9B1C986
:101D600075260AEAF4200102D285300102C285B14B
:101D7000C9C3134002C201D526EB22B17FEAFB2082
:101D80008502A17F308502A184752608AE24AF2587
:101D9000C3EF13FFEE13FEB1CDB1C9C3EA13308513
:101DA000024480FA30E703632201C3E52313F523DD
:101DB000E52213F52250066323A0632201D526D91C
:101DC000E52265236523F52222AE24AF250E0FDE22
:101DD000FEDFFCD20122424C48656C693437316326
:041DE000F3300601D5
:00000001FF
